:100000000C940C040C9453040C9453040C9453045B
:100010000C9453040C9453040C9453040C94530404
:100020000C9453040C9453040C94030E0C94D50EAE
:100030000C9453040C9453040C9453040C945304E4
:100040000C9453040C9455230C9453040C945304B3
:100050000C9453040C94E11C0C9453040C9453041E
:100060000C9453040C9453040C9453040C945304B4
:100070000C9453040C9453040C9453040C945304A4
:100080000C9453040C9453040C9453040C94530494
:100090000C9453040C9453040C9453040C94530484
:1000A0000C9453040C9453040C945304420F640FA7
:1000B0005210640F5210A90FCC0F5210211034109F
:1000C000201320135D135D13A013DE13F715F7152E
:1000D000F713F715F814F814CB15F715F715E21503
:1000E0000262000162026201620035002E003000EF
:1000F0006400015400001E00140004001D000000F4
:1001000006521F001A0016001B00E3002B002000FF
:10011000080007000600E0002C002100150009007F
:100120001900E2000552220017000A000500000035
:10013000000029002A0000004C0000000752470080
:100140003900000053000000000023001C000B00D9
:10015000110000004900240018000D001000E60006
:10016000000025000C000E003600E40028002600E8
:1001700012000F003700E700E500270013003300EE
:100180003800460004522D002F0034003100480092
:100190000000210222021A000800010000003402BF
:1001A0000500040004000000065236020800180092
:1001B0001C00E3002B00370213000C001B00E000C2
:1001C0002C002602120008003700E2000552270228
:1001D000080036000E000000000029002A00000080
:1001E0004C00000007524700390000005300000097
:1001F00000001F02230206003400000049002E0206
:10020000190017001400035200002D00070016000B
:100210000A00E400280038000F0015000B00E7007A
:10022000025225020D0011000900460004522E0062
:100230001D001000060048000000200235001A02D0
:100240000802010000001E00050204020402010071
:1002500001001F00080218021C02E3022B0220000A
:1002600013020C021B02E00201002100120208022C
:100270003302E20201002200080233000E020000F5
:100280000100010001000000010000000100010068
:100290000100000001000000010023001E02060210
:1002A0003802000001002400190217021402E602BD
:1002B00001002500070216020A02E40201002600DE
:1002C0000F0215020B02E702010027000D021102C6
:1002D00009020100010001001D02100206020100D6
:1002E0000000210222021A0008000100000034026E
:1002F00031020400310000000652360208001800E6
:100300002F02E3002B00370224020C003002E00031
:100310002D022F00120022143700E2000552300097
:100320000800360035020000000029002A00000005
:100330004C00000007524700390000005300000045
:1003400000001F02230206003400000049002E02B4
:10035000190017001400010000002D00070016000E
:100360000A00E400280038000F0015000B00E70029
:10037000025225020D0011000900460004522E0011
:100380001D001000060048000000000000000000F2
:100390000000000000003A00000000000000000023
:1003A00000003B00000000000000010000003C00D5
:1003B000000000000000010000003D0000000000FF
:1003C0000000010000003E000000000000000000EE
:1003D000000000000000000000000000000000001D
:1003E000000000000000000000003F0000000000CE
:1003F00000000000000040000000000000000100BC
:100400000000410000000000000001000000420068
:100410000000000000000100010043000000000097
:100420000000000001004400450068006900000071
:1004300000000000000000000000000000000000BC
:1004400000000000000000000000000000000000AC
:10045000000001000000000000000000000001009A
:10046000000000000000000000000100010000008A
:10047000000000000000000000000000000000007C
:10048000000000000000000000000000000000006C
:100490000000000000000000000000000000570005
:1004A0005F005C00590062000000560060005D00C3
:1004B0005A0000305800540061005E005B00850067
:1004C00001005500000000000000000000000000D6
:1004D000000000000000000000000000000000001C
:1004E000000000000000000000000000000000000C
:1004F00001000000000000000000010000000000FA
:1005000000000000000001000000000000000000EA
:1005100000000100000000000000000000000000DA
:1005200000000000000000000000000000000000CB
:1005300000000000000000000000000000000000BB
:1005400000000000000000004A0050000000010010
:1005500000000000520051000000010000000000F7
:100560004D004F0000000100010000004B004E0054
:10057000000000000000000000000000000000007B
:10058000000000000000000000000000000000006B
:10059000000000000000000000000000000000005B
:1005A0000000010000000000000000000000010049
:1005B000000000000000000000000100000000003A
:1005C000000000000000000000000000000000002B
:1005D000000000000100000000000000000000001A
:1005E000000000000000000000000000000000000B
:1005F000F400F2000000010000000000F000F10033
:100600000000010000000000F500F3000000010000
:1006100001000000F900FA000000000000000000E6
:1006200000000000000000000000160345007200FA
:1006300067006F0044006F007800200045005A00FA
:10064000000016034500720067006F0044006F0051
:100650007800200045005A00000004030904090244
:100660006D00040100A0FA0904000001030101006B
:10067000092111010001223F000705810308000A3A
:1006800009040100010301020009211101000122F6
:100690004D000705820308000A0904020001030057
:1006A000000009211101000122360007058303081B
:1006B000000A0904030001030000000921110100E0
:1006C0000122390007058403100001120110010006
:1006D000000008EDFE0713010001020001050109F9
:1006E00006A101050719E029E71500250195087500
:1006F00001810205081901290595057501910295E9
:100700000175039101050719002977150025019549
:100710007875018102C005010980A10185021601D9
:100720000026B7001A01002AB70075109501810054
:10073000C0050C0901A1018503160100269C021ABF
:1007400001002A9C02751095018100C00501090273
:10075000A1010901A10005091901290515002501BB
:100760009505750181029501750381010501093027
:1007700009311581257F9502750881060938158193
:10078000257F950175088106050C0A38021581251B
:100790007F950175088106C0C005010906A1010504
:1007A0000719E029E71500250195087501810295D3
:1007B0000175088101050819012905950575019143
:1007C000029501750391010507190029FF15002500
:1007D000FF950675088100C00000000000000000C1
:1007E000000000010204060A0F17202C3A4A5D712E
:1007F000879DB3C7DAE9F5FCFFFCF5E9DAC7B39DDD
:1008000087715D4A3A2C20170F0A06040201000086
:10081000000000000000000011241FBECFEFDAE04E
:10082000DEBFCDBF04B603FE27C08091EE019091DC
:10083000EF01A091F001B091F1018730904BA740FA
:10084000B04BD1F41092EE011092EF011092F00132
:100850001092F10114BE84B7877F84BF0FB6F8945D
:10086000A89580916000886180936000109260007C
:100870000FBEE0E0FFE3099511E0A0E0B1E0ECE499
:10088000FAE402C005900D92A433B107D9F721E034
:10089000A4E3B1E001C01D92AE3EB207E1F70E94B1
:1008A000440B0C9424250C940000611107C0FC013A
:1008B0008281811106C080EE90E0089580E090E092
:1008C000089583EE90E00895089508950C946504CA
:1008D00056985E9825982D9826982E9827982F98A8
:1008E0008FEF90E0909389008093880090938B0025
:1008F00080938A0090938D0080938C00259A2D9A86
:100900002FEF80E792E0215080409040E1F700C057
:100910000000269A2E9A2FEF80E792E02150804027
:100920009040E1F700C00000279A2F9A2FEF80E750
:1009300092E0215080409040E1F700C000002598EF
:100940002D982FEF80E792E0215080409040E1F712
:1009500000C0000026982E982FEF80E792E02150EB
:1009600080409040E1F700C0000027982F985698EB
:100970005E9825982D9826982E9827982F98089558
:1009800089EA8093800089E08093810024982C98E4
:100990003F988AB18F748AB96E98479A8BB1806BF1
:1009A0008BB9769A0E9468040C94640480E2809368
:1009B00000018091340181110EC00E94250581E063
:1009C000809334012FEF83ED90E3215080409040DD
:1009D000E1F700C0000080E40E942B058093000135
:1009E00081112EC00E94550580930001811128C0FD
:1009F0000E94550580930001811122C08FE30E945F
:100A000055058093000181111BC00E944D0580E4B3
:100A10000E942B0580930001811112C08CE00E947E
:100A200055058093000181110BC00E9455058093EC
:100A30000001811105C08FE30E94550580930001DC
:100A40000E944D058091000108951092B9008AE03E
:100A50008093B800089594EA9093BC009091BC00F4
:100A600097FFFCCF9091B900987F983021F090319A
:100A700011F081E008958093BB0084E88093BC006E
:100A80008091BC0087FFFCCF8091B900887F8831BE
:100A900011F0803471F780E0089584E98093BC0000
:100AA0008091BC0084FDFCCF08958093BB0084E856
:100AB0008093BC008091BC0087FFFCCF9091B9006F
:100AC000987F81E0983209F480E0089584E880936B
:100AD000BC008091BC0087FFFCCF8091BB000895D3
:100AE00080910001811115C080E40E942B05809344
:100AF000000181110CC082E10E9455058093000124
:100B0000811105C08FEF0E945505809300010E945E
:100B10004D0584B1807F84B985B1807F85B98AB164
:100B2000837F8AB98BB1837F8BB93E9846980895AD
:100B30000E94D604809300010E94700580B38C70DF
:100B400080BB81B3836F81BBA6E3B1E0E4E4F1E055
:100B50008EE08E0F11921D928E13FCCF0C94C00468
:100B6000BF92CF92DF92EF92FF920F931F93CF939A
:100B7000DF9380910001882379F0809135018F5FA8
:100B800080933501811108C00E94D6048093000132
:100B9000811102C00E94680406E311E0C0E0D0E0C9
:100BA000DD24D39482E0C82EEE24E394F12CC730E8
:100BB000D10500F580910001811164C080E40E949C
:100BC0002B0580930001811112C082E10E9455051E
:100BD0008093000181110BC0C7010C2E01C0880F4A
:100BE0000A94EAF780950E945505809300010E94BF
:100BF0004D0548C0CA30A1F028F4C83059F0C930BA
:100C000061F005C0CC3089F070F0CD3089F0209AC9
:100C1000289810C0219A29980DC0229A2A980AC0B3
:100C2000239A2B9807C0529A01C0539A5B9802C02E
:100C30003E9A469890EA9A95F1F79FB1799902C049
:100C400082E001C080E091709D25982B7C9902C0C4
:100C500084E001C080E0892B7D9902C038E001C0AA
:100C600030E0832B7E9902C020E101C020E0822B7E
:100C70009FB19095991F9927991F9295990F907EF2
:100C8000892B0FC080910001811149C080E40E942E
:100C90002B0580930001882379F1B12C0E944D052A
:100CA0008B2DF8019081981719F08083C092010173
:100CB0000E94700521960F5F1F4FCE30D10509F0BD
:100CC00076CF80910101882361F1815080930101E9
:100CD000882339F08FE99FE00197F1F700C0000009
:100CE00020C0A4E4B1E0E6E3F1E0CF01825F91919E
:100CF0009D938E13FCCF15C083E10E945505809310
:100D000000018111CACF81E40E942B05809300016C
:100D10008111C3CF0E946605B82EB094BFCF80E08A
:100D2000C0CF0E94660481E0DF91CF911F910F91A7
:100D3000FF90EF90DF90CF90BF900895E82FF0E004
:100D4000EC5BFE4F808108950895089596E0799FA9
:100D5000F001112494E5899FE00DF11D1124E60FA7
:100D6000F11DEE0FFF1FE651FF4F859194910895FD
:100D7000880F991FFC01E659F040859194910895E0
:100D8000880F991FFC01E651FF4F859194910895BA
:100D90000F931F93CF93DF93EC018115904350F590
:100DA000C11580E2D80708F0B3C0CB3BD10590F461
:100DB000C83AD10508F05AC0C53AD10508F04BC071
:100DC000C430D10508F0BCC1219709F0B6C101E0DB
:100DD00010E0F6C1CF3FD10511F008F0B1C1C03F1E
:100DE000D10508F092C0CE01805E9109089708F401
:100DF000A7C1A3C1C11591E5D907A8F4C23020E568
:100E0000D20708F09EC0C11580E5D80709F485C057
:100E100008F091C0C11520E4D20708F08EC1DD278B
:100E20008E01106CCDC1C11580E8D80758F4C115EA
:100E300090E7D90708F07DC1C11520E6D20708F474
:100E400023C17BC1C11580E9D80708F076C1DF70E6
:100E50008E01106AB5C1C53AD10509F473C1C63A0D
:100E6000D10509F072C102E810E4AAC1C83AD1055F
:100E700009F46EC1C93AD10509F46DC1CA3AD10568
:100E800009F46CC1CB3AD10509F46BC1CC3AD10558
:100E900009F46AC1CD3AD10509F469C1C03BD10555
:100EA00009F468C1CE3AD10509F467C1CF3AD1053A
:100EB00009F466C1C13BD10509F465C1C23BD10546
:100EC00009F464C1C33BD10509F463C1C43BD10536
:100ED00009F462C1C53BD10509F461C1C63BD10526
:100EE00009F460C1C73BD10509F45FC1C83BD10516
:100EF00009F45EC1C93BD10509F45DC1CA3BD10506
:100F000009F45CC100E014E45BC18E01106558C1B6
:100F1000CE019F700E94C00654C10E941B169FEF15
:100F200024E38CE0915020408040E1F700C00000B5
:100F30000E94061D45C18091CD0181608093CD0145
:100F40003FC10E94AF1E892B11F40E94951E0E9482
:100F5000CC1E9093EE018093ED01C23090E5D9074D
:100F600021F48091ED01816086C0C43020E5D20774
:100F700021F48091ED0182607EC0C63080E5D80703
:100F800021F48091ED01846076C0C83090E5D907E6
:100F900019F48091ED0127C0CA3020E5D20721F471
:100FA0008091ED01806167C0CC3080E5D80721F4E5
:100FB0008091ED0180625FC0CE3090E5D90721F4C9
:100FC0008091ED01806457C0C03120E5D20721F443
:100FD0008091ED0180684FC0C23180E5D80729F4C7
:100FE0008091ED018460886046C0C33090E5D907E8
:100FF00021F48091ED018E7F3EC0C53020E5D207FF
:1010000021F48091ED018D7F36C0C73080E5D8078F
:1010100021F48091ED018B7F2EC0C93090E5D90776
:1010200019F48091ED0126C0CB3020E5D20721F4E0
:101030008091ED018F7E1FC0CD3080E5D80721F46F
:101040008091ED018F7D17C0CF3090E5D90721F455
:101050008091ED018F7B0FC0C13120E5D20721F4D3
:101060008091ED018F7707C0C331D04531F4809175
:10107000ED018B7F877F8093ED018091ED01909151
:10108000EE010E94D01E9CC08D2F99278F7099274A
:1010900081309105D9F49E012370332702C0880F57
:1010A000991F2A95E2F79C688E0144E0000F111FFA
:1010B0004A95E1F700271370802B912B53E0CC0F5A
:1010C000DD1F5A95E1F7C076DD272FC082309105EC
:1010D00031F4DC2FCC278E01016F106A71C0833090
:1010E000910569F4CE018370992701E010E002C0F8
:1010F000000F111F8A95E2F7C8019C680FC0049782
:1011000009F05EC0CE018370992701E010E002C0B3
:10111000000F111F8A95E2F7C8019A6823E0CC0FEF
:10112000DD1F2A95E1F7C07ED7708C010C2B1D2B9B
:1011300047C0DF708E01106243C000E010E040C085
:101140008E013EC001E810E43BC003E810E438C063
:1011500002EE14E435C009EE14E432C00AEE14E4E1
:101160002FC005EB14E42CC006EB14E429C007EBF8
:1011700014E426C00CEC14E423C00DEC14E420C0ED
:1011800003E815E41DC00AE815E41AC002E915E4F5
:1011900017C004E915E414C001E216E411C003E22B
:1011A00016E40EC004E216E40BC005E216E408C023
:1011B00006E216E405C007E216E402C00AE216E4FD
:1011C000C801DF91CF911F910F91089596E0799F0B
:1011D000F001112494E5899FE00DF11D1124E60F23
:1011E000F11DEE0FFF1FE651FF4F85919491803E58
:1011F0009105E0F4803C910558F58133910509F49F
:101200006FC048F48932910509F463C08A329105B0
:1012100009F46DC072C089339105E9F082389105F7
:10122000D1F08533910509F44DC067C0833E910527
:1012300081F138F4803E9105B9F0823E9105D9F0F4
:101240005CC0863E910561F1873E9105A1F155C0D4
:101250000E94B80608952091ED0120FD02C021FFF3
:101260004CC080EE90E049C08091ED0180FFF9CF45
:1012700089E390E042C08091ED0182FF0EC0809131
:10128000ED0184FF03C080E090E037C083EE90E082
:1012900034C08091ED0182FFF2CF82EE90E02DC04C
:1012A0008091ED0183FF0BC08091ED0184FDEBCFB8
:1012B00087EE90E022C08091ED0183FFF5CF86EEAE
:1012C00090E01BC08091ED0185FF07C089E290E0AE
:1012D00014C08091ED0185FFF9CF85E390E00DC04A
:1012E0008091ED0186FF07C08AE290E006C0809100
:1012F000ED0186FFF9CF81E390E00E94C8060895D2
:1013000008950C948009809162010895CF93DF9332
:1013100000D01F92CDB7DEB79C018091E4018430EC
:1013200019F593E099833B832A839093E9008FEF2B
:101330009091E800815095FD06C095ED9A95F1F7E2
:1013400000008111F5CF8091E80085FF0DC040E0DD
:1013500050E063E070E0CE0101960E94F30B8091B3
:10136000E8008E778093E8000F900F900F90DF9148
:10137000CF910895CF93DF9300D01F92CDB7DEB702
:101380002091E401243021F522E029839B838A8384
:1013900083E08093E9008FEF9091E800815095FD04
:1013A00006C095ED9A95F1F700008111F5CF809177
:1013B000E80085FF0DC040E050E063E070E0CE0142
:1013C00001960E94F30B8091E8008E778093E800ED
:1013D0000F900F900F90DF91CF9108952091E4012D
:1013E0002430F1F422E02093E9002FEF3091E8005F
:1013F000215035FD06C035ED3A95F1F70000211179
:10140000F5CF2091E80025FF0BC040E050E065E0FB
:1014100070E00E94F30B8091E8008E778093E800E3
:101420000895CF93DF93EC019091E401943009F09B
:1014300046C080910C018823D9F080910D0188234A
:10144000B9F09093E9008FEF9091E800815095FDFD
:1014500006C095E19A95F1F700008111F5CF8091D2
:10146000E80085FF2CC040E050E060E170E017C06C
:1014700081E08093E9008FEF9091E800815095FD25
:1014800006C095ED9A95F1F700008111F5CF809196
:10149000E80085FF14C040E050E068E070E0CE0155
:1014A0000E94F30B8091E8008E778093E80080E142
:1014B000FE01A2E5B1E001900D928A95E1F7DF917E
:1014C000CF9108958091E301811109C00E94880D98
:1014D0000E94E50D8091E20084608093E20008950F
:1014E0001092E301089508950C9442230E949C1CDD
:1014F0000E9448230E948B100C94810942E061EC09
:1015000081E00E94020D42E061EC82E00E94020D47
:1015100042E061EC83E00E94020D42E161EC84E074
:101520000C94020D8091E601833009F455C030F42B
:10153000813071F0823009F48EC008958A3009F448
:101540007AC08B3009F460C0893009F09CC020C09B
:101550008091E501813A09F096C08091E800877F8B
:101560008093E8008091E9019091EA01892B21F4B0
:1015700060E182E591E003C060E080E090E070E02F
:101580000E943E0C8091E8008B778093E8000895DC
:101590008091E501813209F076C08091E901909156
:1015A000EA01009719F0039709F06DC08091E800F7
:1015B000877F8093E8008091E80082FD05C08091DC
:1015C000E4018111F8CF5FC08091F1008093620146
:1015D0008091E8008B7753C08091E501813A09F052
:1015E00052C08091E9019091EA01892B09F04BC02A
:1015F0008091E800877F8093E8008091E80080FF79
:10160000FCCF80910C0136C08091E5018132D9F583
:101610008091E9019091EA01892BA9F58091E80078
:10162000877F8093E8000E94370D8091E7018093C7
:101630000C010C941B168091E501813221F58091FB
:10164000E800877F8093E8000E94370D8091E801D1
:101650008093630108958091E501813AA1F480911E
:10166000E800877F8093E8008091E80080FFFCCF4E
:10167000809163018093F1008091E8008E778093E0
:10168000E8000C94370D089584B7877F84BF0FB6A8
:10169000F894A89580916000886180936000109212
:1016A00060000FBE90E080E80FB6F8948093610070
:1016B000909361000FBE0E94DA100E94880D0E9474
:1016C000E50D8091E20084608093E20078940E94AE
:1016D0006B100E94DC1082E091E00E9486100E9454
:1016E00030238091E401853069F40E945A1C809176
:1016F000E2018823B1F30E94881C882391F30E94A1
:10170000DD0BEFCF0E94E210ECCF292F33272330DF
:101710003105C9F064F42130310581F02230310502
:1017200009F043C08DE690E02EE536E042C021325C
:101730003105F1F02232310541F137C082E190E00C
:101740002BEC36E036C099278130910541F082308C
:10175000910541F0892B49F5EAE5F6E005C0E2E4A0
:10176000F6E002C0EAE2F6E0849190E09F0121C039
:101770006430D8F4E62FF0E0EE0FFF1FEE5DFE4F71
:101780002081318189E090E014C0643070F470E011
:10179000FB01EE0FFF1FE65EFE4F20813181FB0152
:1017A000EA5EFE4F808190E004C080E090E020E09F
:1017B00030E0FA0131832083089580E189BD82E120
:1017C00089BD09B400FEFDCF8091D8008F7D809344
:1017D000D8008091E00082608093E0008091E0007A
:1017E00081FDFCCF0895CF92DF92EF92FF920F938D
:1017F0001F93CF93DF93EC018B016A010E94560D7A
:10180000811133C0C114D10439F0F6018081918176
:10181000081B190BC80FD91FE12CF12C011511055C
:1018200019F18091E80085FD16C08091E8008E775F
:101830008093E800C114D10449F0F60180819181C0
:10184000E80EF91EF182E08285E00FC00E94560D7D
:10185000882321F30AC089918093F1000150110976
:10186000FFEFEF1AFF0ADACF80E0DF91CF911F91EF
:101870000F91FF90EF90DF90CF9008952091EB01B2
:101880003091EC012617370748F06115710539F4DE
:101890002091E8002E772093E80001C0B90140E0D4
:1018A00061157105A9F12091E401222309F443C0D7
:1018B000253009F442C02091E80023FD40C020916A
:1018C000E80022FD32C02091E80020FFE9CF4091DE
:1018D000F3002091F20030E0342BFC01CF016115C0
:1018E000710559F02830310540F481918093F10061
:1018F000615071092F5F3F4FF1CF41E02830310532
:1019000009F040E02091E8002E772093E800C8CF4E
:101910004111C9CF0AC08091E401882361F085306C
:1019200061F08091E80083FD0AC08091E80082FFA9
:10193000F2CF80E0089582E0089583E0089581E089
:1019400008952091EB013091EC012617370748F0FC
:101950006115710539F42091E8002E772093E80095
:1019600001C0B901FC0120E06115710591F1809180
:10197000E401882309F440C0853009F43FC0809118
:10198000E80083FD3DC08091E80082FD2FC080917A
:10199000E80080FFE9CF2091F3008091F20090E011
:1019A000922B6115710559F08830910540F424910E
:1019B0002093F1003196615071090196F2CF21E038
:1019C000089709F020E08091E8008E778093E80086
:1019D000CBCF2111CCCF0AC08091E401882361F0E4
:1019E000853061F08091E80083FD0AC08091E800B5
:1019F00082FFF2CF80E0089582E0089583E00895A9
:101A000081E00895982F973058F59093E900981742
:101A100039F07091EC002091ED005091F00003C07E
:101A2000242F762F50E021FF19C03091EB003E7F2C
:101A30003093EB003091ED003D7F3093ED0030911D
:101A4000EB0031603093EB007093EC002093ED00DD
:101A50005093F0002091EE0027FF07C09F5FD3CF87
:101A60008F708093E90081E0089580E0089580916F
:101A7000E50187FF11C08091E80082FD05C08091DB
:101A8000E4018111F8CF11C08091E8008B770BC081
:101A90008091E401882349F08091E80080FFF8CF2D
:101AA0008091E8008E778093E80008952091E4000B
:101AB0003091E50095E64091EC00842F817040FF65
:101AC00022C08091E80080FD1CC08091E401882341
:101AD00091F0853091F08091EB0085FD10C0409130
:101AE000E4005091E5004217530729F39A01915001
:101AF00011F784E0089582E0089583E0089581E07D
:101B0000089580E008954091E80042FFDECF0895F7
:101B10000E94F60D0E94FE0DE0EEF0E080818160F3
:101B20008083E8EDF0E080818F77808319BCA7ED9A
:101B3000B0E08C918E7F8C9380818F7E8083109219
:101B4000E30108950F931F93CF93DF930E94F60D47
:101B50000E94FE0DC8EDD0E088818F778883888150
:101B60008068888388818F7D888319BC1092E40106
:101B70001092E0011092E2011092E10100EE10E0FB
:101B8000F80180818B7F808388818160888342E037
:101B900060E080E00E94020DE1EEF0E080818E7F47
:101BA0008083E2EEF0E080818160808380818860C4
:101BB0008083F80180818E7F808388818061888323
:101BC000DF91CF911F910F910895E8EDF0E08081B2
:101BD0008F7E8083E7EDF0E080818160808384E008
:101BE00082BF81E08093E3010C94A20DE8EDF0E068
:101BF00080818E7F80831092E20008951092DA0037
:101C00001092E10008951F920F920FB60F921124C7
:101C10002F933F934F935F936F937F938F939F93F4
:101C2000AF93BF93EF93FF938091E10082FF0BC0CE
:101C30008091E20082FF07C08091E1008B7F80935A
:101C4000E1000E946A108091DA0080FF1FC080913D
:101C5000D80080FF1BC08091DA008E7F8093DA006D
:101C60008091D90080FF0DC080E189BD82E189BDEE
:101C700009B400FEFDCF81E08093E4010E94620A76
:101C800005C019BC1092E4010E94700A8091E10025
:101C900080FF19C08091E20080FF15C08091E200B2
:101CA0008E7F8093E2008091E20080618093E20069
:101CB0008091D80080628093D80019BC85E0809321
:101CC000E4010E94740A8091E10084FF30C0809199
:101CD000E20084FF2CC080E189BD82E189BD09B4A6
:101CE00000FEFDCF8091D8008F7D8093D800809139
:101CF000E1008F7E8093E1008091E2008F7E8093EF
:101D0000E2008091E20081608093E2008091E00136
:101D1000882311F084E007C08091E30087FD02C0B2
:101D200081E001C083E08093E4010E94760A809103
:101D3000E10083FF29C08091E20083FF25C08091EC
:101D4000E100877F8093E10082E08093E4011092BC
:101D5000E0018091E1008E7F8093E1008091E200BC
:101D60008E7F8093E2008091E20080618093E200A8
:101D700042E060E080E00E94020D8091F000886007
:101D80008093F0000E94730AFF91EF91BF91AF9191
:101D90009F918F917F916F915F914F913F912F9183
:101DA0000F900FBE0F901F9018951F920F920FB6B5
:101DB0000F9211242F933F934F935F936F937F93D1
:101DC0008F939F93AF93BF93CF93DF93EF93FF9343
:101DD000C091E900CF708091EC00D82FD17080FDC8
:101DE000D0E81092E9008091F000877F8093F000A6
:101DF00078940E94190F1092E9008091F000886099
:101E00008093F000CD2BCF70C093E900FF91EF914C
:101E1000DF91CF91BF91AF919F918F917F916F9102
:101E20005F914F913F912F910F900FBE0F901F9098
:101E300018951F93CF93DF93CDB7DEB7AA970FB650
:101E4000F894DEBF0FBECDBFE5EEF1E088E08E0F67
:101E50009091F10091938E13FBCF0E94920A809192
:101E6000E80083FF1FC18091E5019091E601492FB1
:101E700050E04A30510508F015C1FA01EA5AFF4F07
:101E80000C94D924803881F0823809F00BC18091FC
:101E9000E9018F708093E9008091EB0085FB882732
:101EA00080F91092E90006C08091E1019091E20171
:101EB000911182609091E800977F9093E800809361
:101EC000F1001092F100C8C0282F2D7F09F0EAC060
:101ED000882319F0823061F0E5C08091E7018130FC
:101EE00009F0E0C0933009F080E08093E2012BC05C
:101EF0008091E701811127C08091E9018F7009F479
:101F0000D1C08093E9002091EB0020FF1CC09330EA
:101F100021F48091EB00806214C09091EB009061FD
:101F20009093EB0021E030E0A90102C0440F551F5F
:101F30008A95E2F74093EA001092EA008091EB0064
:101F400088608093EB001092E9008091E800877F21
:101F500086C08111A7C01091E7011F778091E3002F
:101F60008078812B8093E3008091E800877F8093C5
:101F7000E8000E94370D8091E80080FFFCCF80913F
:101F8000E30080688093E300111102C082E001C089
:101F900083E08093E40186C08058823008F082C0DC
:101FA0008091E7019091E8018C3D53E0950779F528
:101FB00083E08A838AE289834FB7F894DE0113961F
:101FC00020E03EE051E2E32FF0E050935700E4912F
:101FD00020FF03C0E295EF703F5FEF708E2F90E01F
:101FE000EA3010F0C79601C0C0968D939D932F5F85
:101FF000243149F74FBF8091E800877F8093E80044
:102000006AE270E0CE0101960E943E0C14C0AE015F
:102010004F5F5F4F6091E9010E94850BBC01892BE6
:1020200009F440C09091E800977F9093E80089817F
:102030009A810E94A10C8091E8008B778093E80040
:1020400031C0803879F58091E800877F8093E8007F
:102050008091E0018093F1008091E8008E77809379
:10206000E8000E94370D1EC081111CC09091E7014D
:102070009230C0F48091E800877F8093E8009093CD
:10208000E0010E94370D8091E001811106C080912E
:10209000E30087FD02C081E001C084E08093E40199
:1020A0000E947E0A8091E80083FF0AC08091E800C8
:1020B000877F8093E8008091EB0080628093EB0043
:1020C000AA960FB6F894DEBF0FBECDBFDF91CF91B9
:1020D0001F9108950895CF938091E4018823A1F082
:1020E000C091E900CF709091EC00892F817090FD34
:1020F00080E8C82B1092E9008091E80083FD0E94DF
:10210000190FCF70C093E900CF91089590936901A2
:10211000809368010895E0916801F091690130971A
:1021200021F00190F081E02D099480E00895E09184
:102130006801F0916901309721F00280F381E02D70
:1021400009940895E0916801F0916901309721F0B8
:102150000480F581E02D0994089520916601309165
:1021600067018217930771F090936701809366016E
:10217000E0916801F0916901309721F00680F781C4
:10218000E02D099408952091640130916501821732
:10219000930771F09093650180936401E091680169
:1021A000F0916901309721F00084F185E02D0994C8
:1021B000089508950C94D9100E94A21C0E949805BD
:1021C0000C94681DCF92DF92EF92FF920F931F93B2
:1021D000CF93DF93CDB7DEB72B970FB6F894DEBF62
:1021E0000FBECDBF0E94B0058BE6C82E81E0D82E71
:1021F00000E010E0E02E802F0E949E06F601419143
:102200006F01F42EF826B1F40F5F1F4F0E30110549
:1022100089F78FEF89838A831B820E94AB1C8160C0
:10222000782F9D838C8349815A816B818D810E9497
:10223000851140C09091CD0191FF04C08B870E9411
:10224000A4068B8520E030E04F2D50E0922FBA019C
:10225000022E02C0759567950A94E2F760FF24C0CC
:102260002E83EF8221E030E0690102C0CC0CDD1C3E
:102270009A95E2F790E08C219D21892B09F420E0CA
:1022800028870E94AB1C8160782F9A8789874E81AE
:102290005F8168858A850E948511F801E559FE4FA6
:1022A0008081C826C08206C02F5F3F4F263031058F
:1022B00069F6AACF0E944F2010916A010E948B10EC
:1022C0001817A1F00E948B1080936A012B960FB60D
:1022D000F894DEBF0FBECDBFDF91CF911F910F915C
:1022E000FF90EF90DF90CF900C9481092B960FB662
:1022F000F894DEBF0FBECDBFDF91CF911F910F913C
:10230000FF90EF90DF90CF900895CF93DF93CDB7FC
:10231000DEB72B970FB6F894DEBF0FBECDBF4F834D
:10232000588769877A878B87DE01119686E0FD01E1
:1023300011928A95E9F785E0FE01379601900D929A
:102340008A95E1F749815A816B817C818D819E81DB
:102350000E94B5182B960FB6F894DEBF0FBECDBF06
:10236000DF91CF9108950895CF93882309F4C2C0D7
:10237000C82F823859F40E948B1081FDBBC089E3BD
:102380000E945E1B0E942B1C89E30CC0833879F4E9
:102390000E948B1080FDAEC083E50E945E1B0E94F0
:1023A0002B1C83E50E94A01BCF910C942B1C84381E
:1023B00059F40E948B1082FD9DC087E40E945E1B31
:1023C0000E942B1C87E4EECF8CEF8C0F813A48F4EF
:1023D0008C2F0E94952281118DC08C2F0E945E1B34
:1023E000E3CF80E28C0F883048F4C77081E001C0F1
:1023F000880FCA95EAF70E94E41BD6CF8BE58C0FB5
:10240000833078F4C53A29F0C63A31F083E890E099
:1024100005C081E890E002C082E890E0CF910C9482
:10242000AD1088E58C0F833108F064C0C83A39F1EB
:10243000C93A41F1CA3A49F1CB3A51F1CC3A59F192
:10244000CD3A61F1C03B69F1CE3A71F1CF3A79F101
:10245000C13B81F1C23B89F1C33B91F1C43B99F18E
:10246000C53BA1F1C63BA9F1C73BB1F1C83BB9F1EE
:10247000C93BC1F1CA3BC9F180E090E038C082EEAF
:1024800090E035C089EE90E032C08AEE90E02FC037
:1024900085EB90E02CC086EB90E029C087EB90E0C4
:1024A00026C08CEC90E023C08DEC90E020C083E847
:1024B00091E01DC08AE891E01AC082E991E017C05E
:1024C00084E991E014C081E292E011C083E292E0DD
:1024D0000EC084E292E00BC085E292E008C086E282
:1024E00092E005C087E292E002C08AE292E0CF91DA
:1024F0000C94C310CF910895882309F44BC08238FF
:1025000059F40E948B1081FF45C089E30E945E1B35
:102510000E942B1C89E30CC0833871F40E948B103D
:1025200080FF38C083E50E945E1B0E942B1C83E560
:102530000E94A01B0C942B1C843859F40E948B1011
:1025400082FF28C087E40E945E1B0E942B1C87E448
:10255000EFCF9CEF980F913A58F390E2980F983094
:1025600050F4877091E001C0990F8A95EAF7892F9E
:102570000E94EA1BDFCF9BE5980F933020F480E0A8
:1025800090E00C94AD10885A833120F480E090E004
:102590000C94C3100895882321F00E94E41B0C942E
:1025A0002B1C0895882321F00E94EA1B0C942B1CFD
:1025B0000895BF92CF92DF92EF92FF920F931F93F5
:1025C000CF93DF9300D000D000D0CDB7DEB725E0A9
:1025D000FC01DE01119601900D922A95E1F7FC01B4
:1025E000D08011810281258122952F7043815481F1
:1025F000452B09F4FCC21F3F21F4FFEFDF1609F45D
:10260000F6C27C012E830E94B311D9821A8369819C
:102610007A81802F0E945A1B182FB92E0E940F1BFF
:102620000E94D6192E81002319F00E94011C2E81D0
:10263000EB2DE295EF70F0E0E05AFF4F0C94D924B7
:102640008B2D807F9B2D9F70F92E882319F0F2949B
:1026500080EFF822002389F0FF2009F475C280E2A0
:10266000810F883020F48F2D0E94E41B03C08F2D32
:102670000E94F41B0E942B1C67C2812F0E947C12B7
:10268000FF2009F4B4C2105E8F2D183018F40E9498
:10269000EA1B02C00E94FA1B26960FB6F894DEBF12
:1026A0000FBECDBFDF91CF911F910F91FF90EF90A3
:1026B000DF90CF90BF900C942B1C3B2D307F8B2D47
:1026C0008F70303211F08295807F112319F0113014
:1026D00021F12CC00023B9F0222309F4A0C121303C
:1026E00009F09DC126960FB6F894DEBF0FBECDBF90
:1026F000DF91CF911F910F91FF90EF90DF90CF90DE
:10270000BF900C94141C222319F0213009F46FC2DD
:102710008E830E94171C8E8196C1002321F02230E7
:1027200008F065C27CC1211162C28DC1002321F075
:10273000222309F474C108C2222309F484C119C2F6
:102740002B2D26952695237030E02115310521F09B
:1027500021303105D1F04BC2002321F0812F9B2D78
:10276000937002C080E090E026960FB6F894DEBF2A
:102770000FBECDBFDF91CF911F910F91FF90EF90D2
:10278000DF90CF90BF900C94AD10002321F0812FEB
:102790009B2D937002C080E090E026960FB6F894CF
:1027A000DEBF0FBECDBFDF91CF911F910F91FF9084
:1027B000EF90DF90CF90BF900C94C310812F002337
:1027C00019F00E94571F02C00E94BF1F26960FB625
:1027D000F894DEBF0FBECDBFDF91CF911F910F9157
:1027E000FF90EF90DF90CF90BF900C9444208B2D02
:1027F000837009F07BC00111FAC1812F8295869503
:102800008770880F880F912F9F70C92ED12CE12CD3
:10281000F12C082E04C0CC0CDD1CEE1CFF1C0A940D
:10282000D2F714FF12C04FE050E060E070E004C047
:10283000440F551F661F771F8A95D2F7CB01BA0147
:10284000609570958095909503C060E070E0CB0135
:102850002B2D269526952370422F50E042305105AE
:10286000D9F04330510569F16C297D298E299F29C2
:102870004130510551F126960FB6F894DEBF0FBED8
:10288000CDBFDF91CF911F910F91FF90EF90DF901F
:10289000CF90BF900C94FD196C297D298E299F291A
:1028A00026960FB6F894DEBF0FBECDBFDF91CF9155
:1028B0001F910F91FF90EF90DF90CF90BF900C94FD
:1028C000191A0E94FD19C701B60126960FB6F89491
:1028D000DEBF0FBECDBFDF91CF911F910F91FF9053
:1028E000EF90DF90CF90BF900C94E119002319F086
:1028F0008B2D817001C08695882309F478C1812FC2
:10290000829586958770880F880F912F9F70C92EAA
:10291000D12CE12CF12C082E04C0CC0CDD1CEE1CBB
:10292000FF1C0A94D2F714FF12C04FE050E060E0A1
:1029300070E004C0440F551F661F771F8A95D2F7B9
:10294000CB01BA01609570958095909503C060E0C9
:1029500070E0CB012B2D269526952370422F50E059
:1029600042305105D9F04330510569F16C297D2978
:102970008E299F294130510551F126960FB6F894C2
:10298000DEBF0FBECDBFDF91CF911F910F91FF90A2
:10299000EF90DF90CF90BF900C94D71A6C297D29CF
:1029A0008E299F2926960FB6F894DEBF0FBECDBFA5
:1029B000DF91CF911F910F91FF90EF90DF90CF901B
:1029C000BF900C94F31A0E94D71AC701B60126963D
:1029D0000FB6F894DEBF0FBECDBFDF91CF911F9130
:1029E0000F91FF90EF90DF90CF90BF900C94BB1AA7
:1029F000103FD1F118F4103E50F4A1C0123F09F479
:102A000063C008F44CC0133F09F473C098C01F7032
:102A10008B2D8F710023A1F00E94541A812F2696CE
:102A20000FB6F894DEBF0FBECDBFDF91CF911F91DF
:102A30000F91FF90EF90DF90CF90BF900C94CB124E
:102A40000E94751A812F26960FB6F894DEBF0FBE2E
:102A5000CDBFDF91CF911F910F91FF90EF90DF904D
:102A6000CF90BF900C94D2120023A9F02111BFC0C7
:102A70008B2D8F7126960FB6F894DEBF0FBECDBF9B
:102A8000DF91CF911F910F91FF90EF90DF90CF904A
:102A9000BF900C949A1A223008F0A9C0E9CF002305
:102AA000A9F08B2D8F7126960FB6F894DEBF0FBE5E
:102AB000CDBFDF91CF911F910F91FF90EF90DF90ED
:102AC000CF90BF900C94541A002359F38B2D8F7123
:102AD00026960FB6F894DEBF0FBECDBFDF91CF9123
:102AE0001F910F91FF90EF90DF90CF90BF900C94CB
:102AF000751A002399F08B2D8F7126960FB6F894D6
:102B0000DEBF0FBECDBFDF91CF911F910F91FF9020
:102B1000EF90DF90CF90BF900C943F1A26960FB69F
:102B2000F894DEBF0FBECDBFDF91CF911F910F9103
:102B3000FF90EF90DF90CF90BF900C94351A002358
:102B4000A9F0222309F4ADCF812F26960FB6F89471
:102B5000DEBF0FBECDBFDF91CF911F910F91FF90D0
:102B6000EF90DF90CF90BF900C94B411222309F422
:102B7000ADCF812F26960FB6F894DEBF0FBECDBF26
:102B8000DF91CF911F910F91FF90EF90DF90CF9049
:102B9000BF900C947C124B2D4F70612FC7010E9487
:102BA000550426960FB6F894DEBF0FBECDBFDF9159
:102BB000CF911F910F91FF90EF90DF90CF90BF903A
:102BC0000C9459194B2D4F70612FC70126960FB6E3
:102BD000F894DEBF0FBECDBFDF91CF911F910F9153
:102BE000FF90EF90DF90CF90BF900C94A5062696B3
:102BF0000FB6F894DEBF0FBECDBFDF91CF911F910E
:102C00000F91FF90EF90DF90CF90BF9008950E94BA
:102C1000011C0E94111C0E94D61B0E942B1C0E94AA
:102C2000F4200E94442080E090E00E94AD1080E0FB
:102C300090E00C94C3100E94F11B0C9407160E94A4
:102C40004F1B292F22952F7030E02C3031054CF48A
:102C50002A3031056CF4225031092230310588F4D4
:102C600007C02C30310549F02F30310531F009C053
:102C7000803E48F0803F29F406C093FB882780F906
:102C8000089580E0089581E00895CF93DF9300D008
:102C900000D01F92CDB7DEB70F900F900F900F901E
:102CA0000F90DF91CF910895CF93DF9300D000D0A4
:102CB00000D0CDB7DEB726960FB6F894DEBF0FBEB4
:102CC000CDBFDF91CF9108951F93CF93DF93C09134
:102CD000790116E080917A01C81799F0D0E01C9F25
:102CE000F0011D9FF00D1124E558FE4F40815181E8
:102CF00062817381848195810E9454162196C770E8
:102D0000E9CFDF91CF911F9108954091AB01509190
:102D1000AC016091AD017091AE018091AF019091D5
:102D2000B0010C9454168091B00182958F7009F017
:102D300054C08091AD01882309F44FC0809179017E
:102D4000A0917A016091AB017091AC014091AE010C
:102D50005091AF01B6E08A1709F43FC090E04115E9
:102D60005105C1F17F3F11F46F3FA1F1B89FF00110
:102D7000B99FF00D1124E558FE4F218172132AC02E
:102D80002081621327C02281211124C02381348134
:102D90002417350710F421503109241B350B283C2A
:102DA0003105C0F42091B0012F7020612093B00153
:102DB00026E0289FF001299FF00D1124E058FE4FD6
:102DC00080818F70806180838BEA91E00E94D912AC
:102DD0000C94641601968770BECF0895CF92DF924F
:102DE000EF92FF920F931F93CF93DF93CDB7DEB790
:102DF00062970FB6F894DEBF0FBECDBF8C0185E0A1
:102E0000F801DE011D9601900D928A95E1F7D80137
:102E10004C9111965C91119712966C9112971396A2
:102E2000CD90DC9014973091AB017091AC01809102
:102E3000AE019091AF01009709F46BC17F3F19F487
:102E40003F3F09F466C1E090AD01EE2009F4C0C037
:102E50002091B001C816D90628F0F601E81BF90B3D
:102E6000CF0104C0809590958C0D9D1DFF24F39497
:102E7000883C910578F0F12C207F09F0C6C07C2DAC
:102E8000D98AC88A89890E9445168BEA91E00E94F6
:102E9000D912B1C0822F807F09F046C0751314C0CB
:102EA000341312C0611110C02F7020612093B00143
:102EB0000E9485168BEA91E00E94D9128091B001A0
:102EC000D80115968C932EC0CD2819F15F3F11F4CF
:102ED0004F3FF9F0F62E61111CC0809179012091CD
:102EE0007A0136E0821709F45AC090E0389FF00169
:102EF000399FF00D1124E558FE4F7181571306C01C
:102F00007081471303C07281711103C001968770ED
:102F1000E9CFF62E662309F418C18091B0018160D3
:102F20008093B001F12C11C1751308C0341306C091
:102F3000611104C08091B001D801C3C04D875E8784
:102F40008D859E856A8B0E941F166A898823E1F110
:102F50006623D1F12091B001822F82958F7090E08D
:102F6000029774F08091AB019091AC0198878F83A8
:102F70001986DB86CA862C87CE0107960E94D91255
:102F800086E0F801ABEAB1E001900D928A95E1F795
:102F90000E9493160E948516FF24F394D6C04D8795
:102FA0005E878D859E850E944F1B292F22952F704D
:102FB00030E0223031050CF0BCC09F7009F0B6C083
:102FC000805E883008F4C1C0C8010E94D912E4CFE5
:102FD000C816D90608F453C0F601E81BF90BCF0157
:102FE000883C910508F450C0F12C7C2DD98AC88A00
:102FF00089890E944516EBEAF1E086E0DF011D9227
:103000008A95E9F70E948516A0C0751314C0341381
:1030100012C0611110C08091B001F8018583C80110
:103020000E94D91286E0EBEAF1E0DF011D928A9559
:10303000E9F7FE2C8AC04D875E878D859E856A8B59
:103040000E941F166A89882309F4BECF662309F4FB
:10305000BBCF2091B001822F82958F7090E00297B4
:103060000CF48ECF8091AB019091AC019A8389834F
:103070001B82DD82CC822E83CE0101967FCF80958C
:1030800090958C0D9D1DACCFF62E662309F49CCF38
:1030900075132EC034132CC02091B00120FD1FC029
:1030A000822F82958F70D9F0D80115962C931597A1
:1030B0008F3049F08F5F982F9295907F822F8F707D
:1030C000892B15968C93C8010E94D91286E0F801CD
:1030D000ABEAB1E001900D928A95E1F793CF86E0DB
:1030E000F801ABEAB1E001900D928A95E1F72DC0AD
:1030F0004D875E878D859E850E941F16811140CF6A
:103100008091B00181608093B001C8010E94D91202
:103110001CC0662309F458CF4D875E878D859E8538
:103120000E941F16882309F44FCF2ACF811148CF60
:103130000CC0243031050CF047CF9F7009F440CF0C
:10314000F8019581907F09F03BCF8F2D62960FB6E5
:10315000F894DEBF0FBECDBFDF91CF911F910F91CD
:10316000FF90EF90DF90CF9008951F93CF93DF9360
:10317000CDB7DEB72C970FB6F894DEBF0FBECDBF2C
:103180004F83588769877A878B879C87CE010796FC
:103190000E94EE16882369F08F8198852A853B85E9
:1031A000232BF1F19F3F09F063C08F3F09F060C00E
:1031B00037C086E0FE013796DE01119601900D9230
:1031C0008A95E1F76F817885EA85FB85309741F133
:1031D0007F3F11F46F3F21F120917A0130E0C90166
:1031E0000196877099274091790150E084179507DF
:1031F00009F447C069837A83FD83EC8396E0929F4C
:10320000D001939FB00D1124A558BE4FFE013196F9
:1032100001900D929A95E1F780937A010E946416CD
:1032200016E08091790190917A018917C1F1189F78
:10323000C001112485589E4F0E94EE16882379F113
:10324000E09179011E9FF0011124E558FE4F408165
:10325000518162817381848195810E94541680918D
:10326000790190E001968770992780937901D9CFF1
:103270004F81588569857A858B859C850E94541677
:10328000CFCF0E941B1610927A0110927901EBEABF
:10329000F1E086E0DF011D928A95E9F7C1CF2C9617
:1032A0000FB6F894DEBF0FBECDBFDF91CF911F9157
:1032B0000895EF92FF920F931F93CF93DF938C01AA
:1032C000892B09F46CC0F12CEE24E394E8012196DB
:1032D000F8018491843740F4843008F051C0813083
:1032E00081F0823019F15BC0853709F444C0A8F140
:1032F0009CE7980F903708F052C08F770E947C129D
:1033000041C00E5F1F4FFE01C49180E28C0F8830D8
:1033100048F4C7708E2D01C0880FCA95EAF70E9445
:10332000041C14C08C2F0E94B4112DC00E5F1F4FBF
:10333000FE01C49180E28C0F883058F4C7708E2D46
:1033400001C0880FCA95EAF70E940A1C0E942B1C34
:103350001AC08C2F0E947C1216C00E5F1F4FFE01F8
:10336000C491CC2381F08FE99FE00197F1F700C071
:103370000000C150F6CF0E5F1F4FFE01F49003C056
:103380000E94B4118E018F2D882309F49FCFEFE99D
:10339000FFE03197F1F700C000008150F5CFDF91D9
:1033A000CF911F910F91FF90EF9008950895609332
:1033B000B5017093B6018093B7019093B8010C9456
:1033C00007160F931F930091B5011091B60120913C
:1033D000B7013091B801DC01CB01802B912BA22BDE
:1033E000B32B8093B5019093B601A093B701B0932E
:1033F000B8011F910F910C9407160F931F93009122
:10340000B5011091B6012091B7013091B801DC01EE
:10341000CB0180239123A223B3238093B501909302
:10342000B601A093B701B093B8011F910F910C940E
:1034300007160F931F930091B5011091B6012091CB
:10344000B7013091B801DC01CB0180279127A22779
:10345000B3278093B5019093B601A093B701B093C1
:10346000B8011F910F910C9407161092B1011092A0
:10347000B2011092B3011092B4010C94071641E00E
:1034800050E060E070E004C0440F551F661F771FD6
:103490008A95D2F74093B1015093B2016093B30182
:1034A0007093B4010C94071641E050E060E070E0C6
:1034B00004C0440F551F661F771F8A95D2F780916D
:1034C000B1019091B201A091B301B091B401482B28
:1034D000592B6A2B7B2B4093B1015093B20160931F
:1034E000B3017093B4010C94071641E050E060E022
:1034F00070E004C0440F551F661F771F8A95D2F7EE
:1035000040955095609570958091B1019091B20170
:10351000A091B301B091B401482359236A237B23BE
:103520004093B1015093B2016093B3017093B40121
:103530000C94071641E050E060E070E004C0440FD6
:10354000551F661F771F8A95D2F78091B101909120
:10355000B201A091B301B091B401482759276A275D
:103560007B274093B1015093B2016093B3017093F4
:10357000B4010C9407160F931F930091B1011091A1
:10358000B2012091B3013091B401DC01CB01802B59
:10359000912BA22BB32B8093B1019093B201A093F6
:1035A000B301B093B4011F910F910C9407160F93C0
:1035B0001F930091B1011091B2012091B30130919C
:1035C000B401DC01CB0180239123A223B323809398
:1035D000B1019093B201A093B301B093B4011F91D4
:1035E0000F910C9407160F931F930091B101109146
:1035F000B2012091B3013091B401DC01CB018027ED
:103600009127A227B3278093B1019093B201A09391
:10361000B301B093B4011F910F910C940716089554
:10362000CF92DF92EF92FF920F931F93CF93DF938E
:103630008C01C090B501D090B601E090B701F09038
:10364000B8018091B1019091B201A091B301B09104
:10365000B401C82AD92AEA2AFB2ACFE1D0E0D7014F
:10366000C6010C2E04C0B695A795979587950A9428
:10367000D2F780FF06C0B8018C2F0E94E6080197A0
:1036800021F4219760F780E001C08C2FDF91CF916A
:103690001F910F91FF90EF90DF90CF900895CF93FF
:1036A000DF93EC010E94101BBE010E94E608DF912F
:1036B000CF910895CB010E944F1B089590910C016A
:1036C000992321F090910D01911109C020910E01D3
:1036D00030910F01F90132969FEF40E01FC0982F03
:1036E0009695969596959F3050F5E0910E01F09144
:1036F0000F01E90FF11D877021E030E0A90102C040
:10370000440F551F8A95E2F7CA019181892B818365
:1037100008959F3F39F04F5F4E3041F0519158135B
:10372000F8CF0DC05111F7CF942FF5CF9F3F39F04F
:10373000F901E90FF11D97FDFA9582830895089527
:1037400090910C01992321F090910D01911109C0E4
:1037500020910E0130910F01F9013296205F3F4F09
:103760001FC0982F9695969596959F30F0F4E0910E
:103770000E01F0910F01E90FF11D877021E030E09B
:10378000A90102C0440F551F8A95E2F7CA0180952E
:1037900091818923818308953196E217F30729F0F7
:1037A00090819813F9CF1082F7CF089581E090E0CF
:1037B000E0910E01F0910F01E80FF91F10820196C0
:1037C00080319105A9F708959091CC01892B8093C0
:1037D000CC01089580959091CC0189238093CC01F0
:1037E00008951092CC0108959091CB01892B80937C
:1037F000CB01089580959091CB0189238093CB01D3
:1038000008951092CB0108959091CA01892B80935D
:10381000CA01089580959091CA0189238093CA01B5
:1038200008951092CA0108958093B90108951092E5
:10383000B901089580910E0190910F01FC0131961C
:103840009C01205F3F4F80E0919191118F5FE217C3
:10385000F307D1F70895E0910E01F0910F018091E7
:10386000CC018083E0910E01F0910F019081809155
:10387000CB01892B8083E0910E01F0910F019081A3
:103880008091CA01892B80838091B901882361F0DE
:10389000E0910E01F0910F019081892B80830E94AD
:1038A0001A1C81111092B90180910E0190910F01A3
:1038B0000C9497108091E401843039F11092CE017C
:1038C00020E488E190E00FB6F894A895809360001A
:1038D0000FBE2093600080E00E94810983B7817F42
:1038E000846083BF83B7816083BF7894889583B7F2
:1038F0008E7F83BF0FB6F894A89580916000886191
:1039000080936000109260000FBE0895089508959E
:10391000CF930E94861C0E94B0050E94871CC0E0C5
:103920008C2F0E949E06811104C0CF5FCE30C1F75C
:1039300001C081E0CF9108950E941B160E948B1058
:103940000C94810982E084BD93E095BD9AEF97BD08
:1039500080936E0008952FB7F8948091CF019091D5
:10396000D001A091D101B091D2012FBF0895CF9283
:10397000DF92EF92FF920F931F932FB7F89440912D
:10398000CF015091D0016091D1017091D2012FBF30
:103990006A017B01EE24FF248C0120E030E0C01698
:1039A000D106E206F30610F4415051099A01281B92
:1039B000390BC9011F910F91FF90EF90DF90CF90CD
:1039C00008951F920F920FB60F9211248F939F9319
:1039D000AF93BF938091CF019091D001A091D1017D
:1039E000B091D2010196A11DB11D8093CF0190939A
:1039F000D001A093D101B093D201BF91AF919F911B
:103A00008F910F900FBE0F901F9018950E94880DF8
:103A1000F8942FEF87EA91E6215080409040E1F73B
:103A200000C0000087E090EBDC018093EE019093F2
:103A3000EF01A093F001B093F1019CE088E10FB693
:103A4000F894A895809360000FBE90936000FFCF1C
:103A5000EF92FF920F931F93CF93DF93D82FC0E085
:103A60008C2F0E949E0600E010E0E82EF12CC7018A
:103A7000002E02C0959587950A94E2F780FD06C056
:103A80000F5F1F4F0630110591F709C0602F7C2F83
:103A900080E00E94A606D813F3CF81E004C0CF5F78
:103AA000CE30F1F680E0DF91CF911F910F91FF9022
:103AB000EF900895CF93C82F8CE20E94281D882391
:103AC00021F08C2FCF910C94281D80E0CF91089588
:103AD000CF930E94AF1E811102C00E94951EC5E6C1
:103AE000C15049F00E94B0058FE39CE90197F1F7BE
:103AF00000C00000F5CF89E20E945A1D811113C158
:103B00008AE20E945A1D81110E94951E85E00E9442
:103B10005A1D81110E94061D0E94BA1E8093CD017C
:103B200087E00E945A1D8823A9F18BE10E945A1D4B
:103B3000882351F08091CD0181FB222720F991E06B
:103B4000922790FB81F90EC08EE00E945A1D8823B7
:103B500061F08091CD0182FB222720F991E092272C
:103B600090FB82F98093CD0115C080E10E945A1D1F
:103B70009091CD01882341F093FB222720F981E029
:103B8000822780FB93F904C0892F809580FB90F9F0
:103B90009093CD018091CD010E94BE1E0E94CC1E4B
:103BA0008093ED0180EE0E945A1D882341F08091A0
:103BB000ED01982F909590FB80F98093ED0189E3BA
:103BC0000E945A1D882359F08091ED0181FB222724
:103BD00020F991E0922790FB81F98093ED0182EE2C
:103BE0000E945A1D882359F08091ED0182FB222703
:103BF00020F991E0922790FB82F98093ED0186EE07
:103C00000E945A1D882359F08091ED0183FB2227E1
:103C100020F991E0922790FB83F98093ED0183EEE8
:103C20000E945A1D882359F08091ED0184FB2227C0
:103C300020F991E0922790FB84F98093ED0185E3D0
:103C40000E945A1D882359F08091ED0185FB22279F
:103C500020F991E0922790FB85F98093ED0181E3B3
:103C60000E945A1D882359F08091ED0186FB22277E
:103C700020F991E0922790FB86F98093ED0181E194
:103C80000E945A1D882359F08091ED0187FB22275D
:103C900020F991E0922790FB87F98093ED018091C4
:103CA000ED010E94D01E8091ED0187FB882780F9ED
:103CB00080930D0187E20E945A1DC82F8EE10E9459
:103CC0005A1D8111C2608FE10E945A1D8111C4608A
:103CD00080E20E945A1D8111C86081E20E945A1D33
:103CE0008111C06182E20E945A1D8111C06283E28B
:103CF0000E945A1D8111C06484E20E945A1D8823CB
:103D000011F0C06802C0CC2329F08C2F0E94C71E7E
:103D10006C2F03C00E94C31E682F70E080E090E00B
:103D2000CF910C94D719CF9108956DEE7EEF80E07E
:103D300090E00E940F2560E082E090E00E94012563
:103D400060E083E090E00E94012560E084E090E084
:103D50000E94012560E085E090E00C94012580E060
:103D600090E00E94FB2421E08D3E9E4F09F020E070
:103D7000822F089582E090E00C94F324682F82E073
:103D800090E00C94012583E090E00C94F324682FDC
:103D900083E090E00C94012584E090E00C94F324FF
:103DA000682F84E090E00C9401258091D50180FF7C
:103DB0000BC06091130185E0689FB00111247595D7
:103DC0006795759567952BC081FF09C060911301B8
:103DD00085E0689FB00111247595679520C082FF2A
:103DE00007C06091130185E0689FB001112417C0DE
:103DF0009091D6019923D1F060911201961788F71E
:103E00002091130185E0289F90011124929FA00129
:103E1000939F500D112470E0CA010E94C5246038A0
:103E2000710540F46115710539F002C065E070E07C
:103E3000862F08958FE7089581E008958091D50138
:103E400080FF08C06091110170E0759567957595C8
:103E5000679521C081FF06C06091110170E07595E2
:103E6000679519C082FF04C06091110170E010C015
:103E70009091D6019923C1F0609110019617A0F797
:103E800080911101899FC001112470E00E94C52416
:103E90006038710528F46115710521F0862F0895A9
:103EA0008FE7089581E0089561E070E0F4CF803FEE
:103EB00021F40E94D51E819504C0813F29F40E94FF
:103EC000D51E8093D9010895823F21F40E94D51E0A
:103ED000819504C0833F29F40E94D51E8093D801A8
:103EE0000895893F19F40E941E1F05C08A3F31F4CE
:103EF0000E941E1F81958093DA0108958B3F21F463
:103F00000E941E1F819504C08C3F29F40E941E1F31
:103F10008093DB010895843F21F48091D701816073
:103F200017C0853F21F48091D701826011C0863F80
:103F300021F48091D70184600BC0873F21F48091E8
:103F4000D701886005C0883F31F48091D701806136
:103F50008093D70108958D3F21F48091D501816030
:103F60000BC08E3F21F48091D501826005C08F3F48
:103F700029F48091D50184608093D5010895803F14
:103F800039F48091D90187FF6CC01092D90169C0C2
:103F9000813F29F48091D9011816BCF362C0909139
:103FA000D801823F29F497FF5CC01092D80159C014
:103FB000833F19F41916CCF354C0893F41F4809122
:103FC000DA0118160CF04DC01092DA014AC08A3F8F
:103FD00029F48091DA0187FF44C0F6CF8B3F39F492
:103FE0008091DB0187FF3DC01092DB013AC08C3F1E
:103FF00029F48091DB011816BCF333C0843F21F40F
:104000008091D7018E7F17C0853F21F48091D70121
:104010008D7F11C0863F21F48091D7018B7F0BC02B
:10402000873F21F48091D701877F05C0883F31F415
:104030008091D7018F7E8093D70113C08D3F21F4EB
:104040008091D5018E7F0BC08E3F21F48091D501E8
:104050008D7F05C08F3F29F48091D5018B7F8093A0
:10406000D5018091D80181110EC08091D9018111B3
:104070000AC08091DA01811106C08091DB018111B3
:1040800002C01092D601089587ED91E00E94A2101F
:104090000E94AB1C9093D4018093D30108951F9389
:1040A000CF93DF938091D3019091D4010E94B71CEC
:1040B000AC019091D601992321F02091140130E0B8
:1040C00006C0209115018AE0289F90011124421713
:1040D000530708F485C08091D801C091D901D091CF
:1040E000DA011091DB01811107C0C11175C0D11136
:1040F00073C0111171C074C09F3F19F09F5F9093FE
:10410000D601181624F40E94D51E8093D801809100
:10411000D80187FF05C00E94D51E81958093D801E4
:104120001C1624F40E94D51E8093D9018091D901D8
:1041300087FF05C00E94D51E81958093D9016091AB
:10414000D801662331F1C091D901CC2311F1062E9B
:10415000000C770B880B990B0E94CC2323E333E3ED
:1041600043E35FE30E9430240E9494236093D801CC
:104170006C2FCC0F770B880B990B0E94CC2323E379
:1041800033E343E35FE30E9430240E94942360936F
:10419000D9011D1624F40E941E1F8093DA0180911C
:1041A000DA0187FF05C00E941E1F81958093DA0106
:1041B000111624F40E941E1F8093DB018091DB0105
:1041C00087FF05C00E941E1F81958093DB01DF9150
:1041D000CF911F910C9444209F3F09F08FCF97CF30
:1041E000DF91CF911F910895E7EDF1E085E0DF01C8
:1041F0001D928A95E9F71092D6011092D501089583
:10420000833081F128F4813059F08230D1F0089563
:10421000853009F449C0B8F1863009F456C00895D4
:1042200080911501262F30E0280F311D2F3F3105D9
:1042300024F4680F6093150108958FEF80931501A2
:10424000089580911401262F30E0280F311D2F3F53
:10425000310524F4680F6093140108958FEF809363
:104260001401089580911301262F30E0280F311D8D
:104270002F3F310524F4680F6093130108958FEFE9
:1042800080931301089580911201262F30E0280FAA
:10429000311D2F3F310524F4680F609312010895FA
:1042A0008FEF80931201089580911101262F30E045
:1042B000280F311D2F3F310524F4680F6093110141
:1042C00008958FEF80931101089580911001262F9A
:1042D00030E0280F311D2F3F310524F4680F609323
:1042E000100108958FEF809310010895833011F12C
:1042F00028F4813049F0823091F00895853081F1C1
:1043000020F18630C1F1089580911501681720F4DD
:10431000861B8093150108951092150108958091D0
:104320001401681720F4861B8093140108951092DD
:104330001401089580911301681720F4861B80935F
:1043400013010895109213010895809112016817C6
:1043500020F4861B80931201089510921201089593
:1043600080911101681720F4861B80931101089534
:1043700010921101089580911001681720F4861B96
:104380008093100108951092100108950F931F93C8
:104390008D3109F46AC008F03FC08E3009F484C042
:1043A000C0F4873009F46DC068F4863009F0B5C0F8
:1043B0008091CD01817F8E7F8093CD0181E08093BC
:1043C000DD01ACC0883009F457C08B3009F46AC0F5
:1043D000A4C0863109F466C078F4803109F477C04E
:1043E000813109F09AC00E941B1690910D0181E065
:1043F000892780930D0156C0893109F453C08B3150
:1044000009F08BC08091CD0181FB222720F991E03A
:10441000922790FB81F951C0853309F475C048F4A7
:10442000873209F471C008F45EC0893209F46CC0A7
:1044300074C0833430F48A3308F053C0883391F168
:104440006CC0833409F460C0883409F066C00E94EF
:104450001B160FEF13ED20E3015010402040E1F751
:1044600000C000000E94061D1DC00E944E230E9435
:104470008B100E94810916C00E94BA1E0E94CC1E99
:1044800011C09091CD01892F8095817080FB90F9AA
:1044900029F0966098609093CD0140C0997F977FF6
:1044A0009093CD0181E03AC08091CD0182FB22271B
:1044B00020F991E0922790FB82F98093CD01992316
:1044C00089F38091CD0181608093CD01EBCF809104
:1044D000CD0183FB222720F991E0922790FB83F9FD
:1044E000ECCF895301C08D5141E050E060E070E0B5
:1044F0008A019B0104C0000F111F221F331F8A95E0
:10450000D2F7C901B80104C061E070E080E090E03A
:104510000E94D7190E941B16C5CF80E01F910F91F2
:10452000089580E0089580E00895CF93C82F80918A
:10453000DD01813079F018F08230E9F187C0E09137
:104540000E01F0910F018081813169F0823209F012
:104550007FC009C0E0910E01F0910F01808181318F
:1045600011F0823261F48C2F0E949122811104C0DB
:104570008C2F0E94C6211DC081E090E01AC08C2FB4
:104580000E949322811114C0C43179F048F4CB30D9
:1045900079F0C03109F060C082E08093DD0108C08D
:1045A000C93219F0C83321F057C01092DD0154C050
:1045B00081E0817053C0C93289F118F5C43171F1BD
:1045C000A8F4C73009F046C08AE08093150194E151
:1045D0009093140193E0909313018093120188E06B
:1045E0008093110188E28093100134C0CE51C6300F
:1045F00088F5EC2FF0E0E65DFE4F80818093DC01D2
:1046000029C0CE34E9F020F4CB3421F56AE013C0A0
:10461000C13579F0C235F1F461E00DC08091DC0163
:10462000882319F01092DC0115C081E08093DD0130
:1046300015C061E006C08091DC010E9400210AC023
:104640006AE08091DC010E94762104C01092DD01B5
:1046500080E004C081E002C080E0ABCFCF9108953C
:10466000E1E8F0E0808188608083808181608083E0
:104670008FB7F89493E09093890090ED9093880021
:104680008FBF0895EFE6F0E0808182608083089517
:10469000EFE6F0E080818D7F80830895EFE6F0E023
:1046A000908182E08927808308951F920F920FB630
:1046B0000F9211242F933F934F935F936F937F93A8
:1046C0008F939F93AF93BF93EF93FF938091DE01FE
:1046D0009091DF0101969093DF018093DE018111BB
:1046E00003C082E00E948109E091DF01E695E69532
:1046F000F0E0E852F84FE4918091DE018E1303C0A0
:1047000080E00E948109FF91EF91BF91AF919F914D
:104710008F917F916F915F914F913F912F910F906A
:104720000FBE0F901F9018950E949B236894B111A3
:104730000C942A2408950E940F2488F09F5798F023
:10474000B92F9927B751B0F0E1F0660F771F881F96
:10475000991F1AF0BA95C9F714C0B13091F00E94B0
:104760002924B1E008950C942924672F782F8827F5
:10477000B85F39F0B93FCCF3869577956795B395D7
:10478000D9F73EF490958095709561957F4F8F4F46
:104790009F4F0895E89409C097FB3EF4909580954B
:1047A000709561957F4F8F4F9F4F9923A9F0F92FF7
:1047B00096E9BB279395F695879577956795B79575
:1047C000F111F8CFFAF4BB0F11F460FF1BC06F5F5B
:1047D0007F4F8F4F9F4F16C0882311F096E911C06D
:1047E000772321F09EE8872F762F05C0662371F08E
:1047F00096E8862F70E060E02AF09A95660F771FA2
:10480000881FDAF7880F9695879597F9089557FDD1
:104810009058440F551F59F05F3F71F04795880F2E
:1048200097FB991F61F09F3F79F0879508951216C5
:1048300013061406551FF2CF4695F1DF08C0161671
:1048400017061806991FF1CF869571056105089422
:104850000895E894BB2766277727CB0197F9089539
:104860000E9443240C94B4240E94A62438F00E9491
:10487000AD2420F0952311F00C949D240C94A324D6
:1048800011240C942A240E94072470F3959FC1F3ED
:10489000950F50E0551F629FF001729FBB27F00DEE
:1048A000B11D639FAA27F00DB11DAA1F649F662743
:1048B000B00DA11D661F829F2227B00DA11D621F92
:1048C000739FB00DA11D621F839FA00D611D221F4C
:1048D000749F3327A00D611D231F849F600D211D30
:1048E000822F762F6A2F11249F5750409AF0F1F0B3
:1048F00088234AF0EE0FFF1FBB1F661F771F881F1C
:1049000091505040A9F79E3F510580F00C949D2492
:104910000C942A245F3FE4F3983ED4F38695779570
:104920006795B795F795E7959F5FC1F7FE2B880FC1
:10493000911D9695879597F9089597F99F6780E857
:1049400070E060E008959FEF80EC089500240A94E1
:104950001616170618060906089500240A9412165A
:104960001306140605060895092E0394000C11F48D
:10497000882352F0BB0F40F4BF2B11F460FF04C03A
:104980006F5F7F4F8F4F9F4F089597FB072E16F451
:10499000009407D077FD09D00E94DF2407FC05D0E2
:1049A0003EF4909581959F4F0895709561957F4F46
:1049B0000895EE0FFF1F0590F491E02D0994AA1BB6
:1049C000BB1B51E107C0AA1FBB1FA617B70710F0FA
:1049D000A61BB70B881F991F5A95A9F7809590952C
:1049E000BC01CD010895F999FECF92BD81BDF89A21
:1049F000992780B50895A8E1B0E042E050E00C941A
:104A00001625262FF999FECF1FBA92BD81BD20BD74
:104A10000FB6F894FA9AF99A0FBE019608950E947B
:104A20000125272F0C940225DC01CB01FC01F9990B
:104A3000FECF06C0F2BDE1BDF89A319600B40D92EA
:0C4A400041505040B8F70895F894FFCFA3
:104A4C0020028309110AEE09BA0986090101BA018B
:104A5C0028080A03140A3F4D363999074C071607E4
:104A6C00DD0670068906A206BB06010203040506D4
:044A7C00070809001E
:00000001FF
